:020000040800F2
:1000000000000524B5130008C1110008C311000841
:10001000C5110008C7110008C91100080000000040
:10002000000000000000000000000000CB110008EC
:10003000CD11000800000000CF110008D111000808
:10004000051400080514000805140008051400082C
:10005000051400080514000805140008051400081C
:10006000051400080514000805140008051400080C
:1000700005140008051400080514000805140008FC
:10008000051400080514000805140008D91100081B
:1000900005140008E91100080514000805140008FB
:1000A00005140008051400080514000805140008CC
:1000B00005140008051400080514000805140008BC
:1000C00005140008051400080514000805140008AC
:1000D00005140008F91100080514000805140008AB
:1000E00005140008051400080000000005140008AD
:1000F000051400080514000805140008051400087C
:10010000051400080514000805140008051400086B
:10011000051400080514000805140008051400085B
:10012000051400080514000805140008051400084B
:10013000051400080514000805140008051400083B
:1001400000000000000000000000000000000000AF
:10015000051400080514000805140008051400081B
:10016000051400080514000805140008051400080B
:10017000051400080514000805140008000000001C
:1001800005140008051400080514000805140008EB
:1001900005140008051400080514000805140008DB
:1001A00005140008051400080514000800000000EC
:1001B00005140008051400080514000805140008BB
:1001C00005140008051400080000000000000000ED
:1001D00000000000000000000514000800000000FE
:1001E000000000000000000000000000000000000F
:1001F00000000000000000000514000805140008BD
:10020000051400080514000800000000051400088B
:10021000051400080514000805140008051400085A
:10022000051400080000000005140008000000008C
:10023000051400080514000800000000051400085B
:10024000051400080514000805140008051400082A
:10025000051400080514000805140008051400081A
:10026000051400080514000805140008051400080A
:10027000051400080514000805140008000000001B
:1002800005140008051400080514000805140008EA
:10029000000000000514000805140008000000001C
:1002A00000000000051400080514000805140008EB
:1002B00005140008051400080514000805140008BA
:0C02C000051400080514000805140008CF
:1002CC0010B5054C237833B9044B13B10448AFF384
:1002DC0000800123237010BD3C04002400000000AA
:1002EC00CC5E000808B5034B1BB103490348AFF3C0
:1002FC00008008BD0000000040040024CC5E000813
:10030C0080F0004002E000BF81F0004142001FBFBE
:10031C005FEA410392EA030F7FEA226C7FEA236CC7
:10032C006AD04FEA1262D2EB1363C1BFD2184140BC
:10033C0048404140B8BF5B42192B88BF704710F052
:10034C00004F40F4000020F07F4018BF404211F0F5
:10035C00004F41F4000121F07F4118BF494292EA5D
:10036C00030F3FD0A2F1010241FA03FC10EB0C0089
:10037C00C3F1200301FA03F100F0004302D5494216
:10038C0060EB4000B0F5000F13D3B0F1807F06D3C3
:10039C0040084FEA310102F10102FE2A51D2B1F1BB
:1003AC00004F40EBC25008BF20F0010040EA0300B0
:1003BC007047490040EB0000013A28BFB0F5000F30
:1003CC00EDD2B0FA80FCACF1080CB2EB0C0200FAE6
:1003DC000CF0AABF00EBC25052421843BCBFD04035
:1003EC001843704792F0000F81F4000106BF80F4AF
:1003FC0000000132013BB5E74FEA41037FEA226C72
:10040C0018BF7FEA236C21D092EA030F04D092F03C
:10041C00000F08BF0846704790EA010F1CBF002070
:10042C00704712F07F4F04D1400028BF40F00040CD
:10043C00704712F100723CBF00F50000704700F0ED
:10044C00004343F0FE4040F4000070477FEA226214
:10045C0016BF08467FEA23630146420206BF5FEAE5
:10046C00412390EA010F40F4800070474FF00003E5
:10047C0004E000BF10F0004348BF40425FEA000CAC
:10048C0008BF704743F0964301464FF000001CE054
:10049C0050EA010208BF70474FF000030AE000BFAA
:1004AC0050EA010208BF704711F0004302D54042E8
:1004BC0061EB41015FEA010C02BF8446014600205A
:1004CC0043F0B64308BFA3F18053A3F50003BCFA75
:1004DC008CF2083AA3EBC25310DB01FA02FC634422
:1004EC0000FA02FCC2F12002BCF1004F20FA02F229
:1004FC0043EB020008BF20F00100704702F120021C
:10050C0001FA02FCC2F1200250EA4C0021FA02F27C
:10051C0043EB020008BF20EADC7070474FF0FF0C81
:10052C001CEAD0521EBF1CEAD15392EA0C0F93EA7C
:10053C000C0F6FD01A4480EA010C400218BF5FEA1E
:10054C0041211ED04FF0006343EA501043EA511191
:10055C00A0FB01310CF00040B1F5000F3EBF49008B
:10056C0041EAD3715B0040EA010062F17F02FD2A8F
:10057C001DD8B3F1004F40EBC25008BF20F0010072
:10058C00704790F0000F0CF0004C08BF49024CEA89
:10059C00502040EA51207F3AC2BFD2F1FF0340EA1B
:1005AC00C250704740F400004FF00003013A5DDC8C
:1005BC0012F1190FDCBF00F000407047C2F10002CD
:1005CC00410021FA02F1C2F1200200FA02FC5FEABA
:1005DC00310040F1000053EA4C0308BF20EADC7004
:1005EC00704792F0000F00F0004C02BF400010F476
:1005FC00000F013AF9D040EA0C0093F0000F01F023
:10060C00004C02BF490011F4000F013BF9D041EA44
:10061C000C018FE70CEAD15392EA0C0F18BF93EA46
:10062C000C0F0AD030F0004C18BF31F0004CD8D170
:10063C0080EA010000F00040704790F0000F17BFF7
:10064C0090F0004F084691F0000F91F0004F14D03D
:10065C0092EA0C0F01D142020FD193EA0C0F03D195
:10066C004B0218BF084608D180EA010000F0004098
:10067C0040F0FE4040F40000704740F0FE4040F473
:10068C00400070474FF0FF0C1CEAD0521EBF1CEA12
:10069C00D15392EA0C0F93EA0C0F69D0A2EB030230
:1006AC0080EA010C49024FEA402037D04FF08053CA
:1006BC0043EA111143EA10130CF000408B4238BF8F
:1006CC005B0042F17D024FF4000C8B4224BF5B1A9D
:1006DC0040EA0C00B3EB510F24BFA3EB510340EAEB
:1006EC005C00B3EB910F24BFA3EB910340EA9C0099
:1006FC00B3EBD10F24BFA3EBD10340EADC001B0109
:10070C0018BF5FEA1C1CE0D1FD2A3FF650AF8B42AC
:10071C0040EBC25008BF20F0010070470CF0004CB9
:10072C004CEA50207F32C2BFD2F1FF0340EAC250E4
:10073C00704740F400004FF00003013A37E792F0A5
:10074C00000F00F0004C02BF400010F4000F013A03
:10075C00F9D040EA0C0093F0000F01F0004C02BFFE
:10076C00490011F4000F013BF9D041EA0C0195E767
:10077C000CEAD15392EA0C0F08D142027FF47DAF00
:10078C0093EA0C0F7FF470AF084676E793EA0C0FF0
:10079C0004D14B023FF44CAF08466EE730F0004CEE
:1007AC0018BF31F0004CCAD130F000427FF45CAF7E
:1007BC0031F000437FF43CAF5FE700BF42000ED244
:1007CC00B2F1FE4F0BD34FF09E03B3EB126209D480
:1007DC004FEA002343F0004323FA02F070474FF036
:1007EC000000704712F1610F01D1420202D14FF0AB
:1007FC00FF3070474FF00000704700BF53B94AB943
:10080C00002908BF00281CBF4FF0FF314FF0FF300C
:10081C0000F06CB9ADF1080C6DE904CE00F006F8EF
:10082C00DDF804E0DDE9022304B070472DE9F04760
:10083C00089E0D4604468E46002B40F082808A426C
:10084C00174646D9B2FA82F24AB1C2F1200105FA32
:10085C0002F320FA01F1974041EA030E94404FEA6B
:10086C001748230CBEFBF8FCB9B208FB1CEE43EA9C
:10087C000E430CFB01F098420AD9FB180CF1FF3522
:10088C0080F01681984240F21381ACF1020C3B448B
:10089C001B1AA4B2B3FBF8F008FB103344EA034470
:1008AC0000FB01F1A14209D93C1900F1FF3380F0A2
:1008BC000181A14240F2FE8002383C44641A40EAB5
:1008CC000C4000211EB1D4400023C6E90043BDE812
:1008DC00F08702B9FFDEB2FA82F2002A4FD1CB1BAD
:1008EC004FEA174E1FFA87F80121B3FBFEFC250CCB
:1008FC000EFB1C3345EA034508FB0CF3AB4207D94E
:10090C007D190CF1FF3002D2AB4200F2E780844635
:10091C00ED1AA3B2B5FBFEF00EFB105543EA0544ED
:10092C0008FB00F8A04507D93C1900F1FF3302D2AF
:10093C00A04500F2D7801846A4EB080440EA0C400E
:10094C00C0E78B4208D9002E00F0AF800021C6E929
:10095C0000050846BDE8F087B3FA83F100294BD1B6
:10096C00AB4202D3824200F2B780841A65EB0303D8
:10097C0001209E46002EAAD0C6E9004EA7E7C2F180
:10098C00200C01FA02F3974020FA0CF04FEA174EB4
:10099C0021FA0CFC1843BCFBFEF1050C0EFB11CC30
:1009AC001FFA87F845EA0C4501FB08F3AB4204FA41
:1009BC0002F409D97D1901F1FF3C80F08B80AB4228
:1009CC0040F2888002393D44EB1A85B2B3FBFEF04D
:1009DC000EFB103345EA034500FB08F3AB4207D985
:1009EC007D1900F1FF3C71D2AB426FD902383D4406
:1009FC00EB1A40EA014178E7C1F1200C8B4022FA56
:100A0C000CF71F4320FA0CF405FA01F34FEA174ECA
:100A1C0025FA0CF51C43230CB5FBFEF91FFA87F8DD
:100A2C000EFB195543EA054509FB08FAAA4502FADB
:100A3C0001F200FA01F308D97D1909F1FF3047D210
:100A4C00AA4545D9A9F102093D44A5EB0A05A4B272
:100A5C00B5FBFEF00EFB105544EA054400FB08F80C
:100A6C00A04507D93C1900F1FF352DD2A0452BD953
:100A7C0002383C4440EA0940A4EB0804A0FB02897C
:100A8C004C45C6464D4619D316D05EB1B3EB0E029B
:100A9C0064EB050404FA0CFCCA404CEA0202CC409C
:100AAC00C6E900240021BDE8F087314630460EE748
:100ABC00AC46EDE6184601E74345E6D2B8EB020E2C
:100ACC0069EB07050138E0E72846D3E760468FE776
:100ADC008146BAE7614677E708464BE7ACF1020C72
:100AEC003D4415E702383C4426E700BF704700BF81
:100AFC00844641EA000313F003036DD1403A41D31D
:100B0C0051F8043B40F8043B51F8043B40F8043BDB
:100B1C0051F8043B40F8043B51F8043B40F8043BCB
:100B2C0051F8043B40F8043B51F8043B40F8043BBB
:100B3C0051F8043B40F8043B51F8043B40F8043BAB
:100B4C0051F8043B40F8043B51F8043B40F8043B9B
:100B5C0051F8043B40F8043B51F8043B40F8043B8B
:100B6C0051F8043B40F8043B51F8043B40F8043B7B
:100B7C0051F8043B40F8043B51F8043B40F8043B6B
:100B8C00403ABDD2303211D351F8043B40F8043B0B
:100B9C0051F8043B40F8043B51F8043B40F8043B4B
:100BAC0051F8043B40F8043B103AEDD20C3205D31B
:100BBC0051F8043B40F8043B043AF9D2043208D013
:100BCC00D2071CBF11F8013B00F8013B01D30B8885
:100BDC0003806046704700BF082A13D38B078DD063
:100BEC0010F003038AD0C3F10403D21ADB071CBF35
:100BFC0011F8013B00F8013B80D331F8023B20F89F
:100C0C00023B7BE7043AD9D3013A11F8013B00F8D7
:100C1C00013BF9D20B7803704B7843708B7883705F
:100C2C006046704770B58AB0002302930393022686
:100C3C0004960124059406930793094D02A92846AE
:100C4C0001F022FA0094234632463146284601F040
:100C5C005DFA22462146284601F073FA0AB070BDAF
:100C6C005804002410B5FFF7DDFF054C204601F0B9
:100C7C0097FA4FF470620349204601F031FC10BD25
:100C8C0058040024020A801B2DE9F04704460B4649
:100C9C00002942D1042A04D8DFE802F03907272DB5
:100CAC0033000026B146B24604E019264FF0AE09D7
:100CBC004FF0020A0021A1600A251D274FF0010800
:100CCC00012B31D0204601F0D1FAC4F814A0C4F89D
:100CDC001C902662A661C4F82480E7622563A56295
:100CEC00204601F087F8BDE8F08714264FF08B09F9
:100CFC004FF0020ADEE714264FF08B094FF0010A81
:100D0C00D8E714264FF03B094FF0010AD2E714261E
:100D1C004FF08B094FF0040ACCE700252F46A8466C
:100D2C002E46A946AA46CBE7053A042A08D8DFE89E
:100D3C0002F01F0310151A00062519274FF00108A1
:100D4C004FF44073A36014264FF03B094FF0010A97
:100D5C00B8E7052513274FF00108F1E705250E2705
:100D6C004FF00108ECE702250D274FF00108E7E7EB
:100D7C000A251D274FF00108E2E700B58BB0019161
:100D8C00002102910391082B00D804930C2B1CD04A
:100D9C00102B1DD0142B1ED0182B1FD0202B20D085
:100DAC00302B21D0402B22D0002305934FF48011FF
:100DBC0006914FF4001107910893099301A901F0D2
:100DCC006AFAB8B90BB05DF804FB09210491DFE7AE
:100DDC000A210491DEE70B210491DDE70C2104913B
:100DEC00DCE70D210491DBE70E210491DAE70F23F8
:100DFC000493D9E70120E5E730B58BB00C461346D8
:100E0C006A46402101F082FA18B1002528460BB041
:100E1C0030BD009B2380039B082B00D8DDB2092B2F
:100E2C0000D80C250A2B00D810250B2B00D8142524
:100E3C000C2B00D818250D2B00D820250E2B00D8F4
:100E4C0030250F2BE2D84025E0E7000008B5034B16
:100E5C00834200D008BD04F047FEFBE75804002491
:100E6C0008B511F0007F04D00268936923F00103E8
:100E7C00936111F4000F00D108BD00F003F8FFF7E7
:100E8C00F1FEF9E708B51548154B036000238360A4
:100E9C00C36003744374837418224261012282611B
:100EAC000221C161016242628262C26202634363D7
:100EBC008263C36320210164042242648364C2649C
:100ECC00036542658365C36501664366826600F00F
:100EDC0091FF00B908BD00F0CBF8FBE758040024E3
:100EEC0000A0004010B5B6B00446002131913291FB
:100EFC00339134913591B82202A804F021FF226875
:100F0C00264B9A4201D036B010BD4FF4004200235C
:100F1C00CDE902234FF080531D9302A802F02AFD65
:100F2C00002837D11E4BD3F8EC2042F48072C3F862
:100F3C00EC20D3F8EC2002F480720092009AD3F8E3
:100F4C00E02042F00102C3F8E020D3F8E03003F0D7
:100F5C0001030193019B4FF4C0533193022332934D
:100F6C000024339434940923359331A90D4801F0AE
:100F7C009FFC22462146132000F0CEFA132000F0ED
:100F8C00FDFA22462146152000F0C6FA152000F085
:100F9C00F5FAB8E700F06CF8C4E700BF00A0004019
:100FAC00004402580000025808B502680B4B9A42E4
:100FBC0000D008BD0A4AD2F8EC3023F48073C2F892
:100FCC00EC304FF4C051074801F062FD132000F0E3
:100FDC00E3FA152000F0E0FAEBE700BF00A00040B8
:100FEC00004402580000025830B589B00024039424
:100FFC0004940594069407941B4BD3F8E02042F01C
:10100C008002C3F8E020D3F8E02002F080020092C6
:10101C00009AD3F8E02042F00102C3F8E020D3F8A4
:10102C00E02002F001020192019AD3F8E02042F094
:10103C000202C3F8E020D3F8E03003F0020302937D
:10104C00029B0A4D22468021284601F0C5FD8023D3
:10105C000393012304930594069403A9284601F0F5
:10106C0027FC09B030BD00BF0044025800000258F4
:10107C0072B6FEE710B59CB04C22002109A804F012
:10108C005FFE2022002101A804F05AFE022001F08C
:10109C00A9FD00230093204B9A6922F440429A61E7
:1010AC009B6903F440430093009B1B4B9B6913F417
:1010BC00005FFAD00222099201200C9040230D937C
:1010CC00129200231393042114911E24159416904C
:1010DC00179118920C2219921A931B9309A801F0DC
:1010EC00ABFDA0B93F23019303210291002303938D
:1010FC00082304934023059306934FF480620792D0
:10110C00089301A802F09AF918B91CB010BDFFF7AA
:10111C00AFFFFFF7ADFF00BF0048025800B583B02A
:10112C0000F094F9FFF7A6FFFFF75EFFFFF7AAFEAA
:10113C0000F0B0F8144D042200212846FFF7A4FD5E
:10114C00FFF790FD04F01EFB0A2000F0BFF90F4CD6
:10115C0000230193009301220A21208804F088FDCA
:10116C002146284604F05EFD642000F0AFF90A2108
:10117C00208804F0A3FD642000F0A8F94FF47A70E5
:10118C0000F0A4F9FEE700BF5804002490050024E9
:10119C0082B0074BD3F8F42042F00202C3F8F420DB
:1011AC00D3F8F43003F002030193019B02B07047B3
:1011BC0000440258FEE7FEE7FEE7FEE7FEE7704755
:1011CC007047704708B500F06FF908BD08B50248C4
:1011DC0001F0DEF908BD00BF5804002408B5024830
:1011EC0001F0D6F908BD00BF5804002408B5024828
:1011FC0003F0A6FB08BD00BFF80400241E4B1B68BF
:10120C0003F00F03062B06D81B4A136823F00F03B9
:10121C0043F007031360194B1A6842F001021A607D
:10122C0000221A611968164A0A401A60124B1B6890
:10123C0013F0080F06D0104A136823F00F0343F085
:10124C00070313600D4B00229A61DA611A620D4993
:10125C0099620D49D9620D4919635A639963DA632E
:10126C0019645A64196821F4802119601A66084BB4
:10127C0043F2D2021A607047002000520044025818
:10128C007FEDF6EA000202020000FF01800201017C
:10129C000040005208B51748174B03604FF4E13378
:1012AC00436000238360C36003610C22426183614D
:1012BC00C36103624362836204F09FF970B9002139
:1012CC000C4804F015FA60B900210A4804F035FA0C
:1012DC0050B9084804F0EDF948B908BDFFF7C8FE4D
:1012EC00EDE7FFF7C5FEEFE7FFF7C2FEF1E7FFF70B
:1012FC00BFFEF2E7F80400240010014010B5B6B0B0
:10130C000446002131913291339134913591B822B8
:10131C0002A804F015FD2268204B9A4201D036B089
:10132C0010BD01220023CDE902230023209302A843
:10133C0002F020FB78BB1A4BD3F8F02042F01002DD
:10134C00C3F8F020D3F8F02002F010020092009ABB
:10135C00D3F8E02042F00202C3F8E020D3F8E030EA
:10136C0003F002030193019B4FF44043319302239A
:10137C0032930024339434940423359331A90948CF
:10138C0001F096FA22462146252000F0C5F82520CA
:10139C0000F0F4F8C3E7FFF76BFECCE70010014058
:1013AC000044025800040258DFF834D0FFF726FF3F
:1013BC000C480D490D4A002302E0D458C4500433A4
:1013CC00C4188C42F9D30A4A0A4C002301E013607A
:1013DC000432A242FBD304F08FFCFFF79FFE704750
:1013EC0000000524000000243C040024905F000849
:1013FC003C04002454100024FEE70000104B1B7822
:10140C000BB90120704710B504464FF47A70B0FB4D
:10141C00F3F30C4A1068B0FBF3F000F0CFF868B9A6
:10142C000F2C01D901200AE0002221464FF0FF3099
:10143C0000F072F8044B1C60002000E0012010BD8D
:10144C0008000024000000240C00002410B5032028
:10145C0000F050F801F0E6FE0F498B69C3F303234B
:10146C000E4AD35C03F01F03D8408B6903F00F03C3
:10147C00D35C03F01F0320FA03F3094A1360094BF2
:10148C0018600F20FFF7BAFF10B10124204610BDE1
:10149C000446FFF77DFEF9E700440258305F000870
:1014AC000400002400000024034B1B78034A11683D
:1014BC000B441360704700BF080000248C05002407
:1014CC00014B1868704700BF8C05002438B50446E2
:1014DC00FFF7F6FF0546B4F1FF3F02D0044B1B7833
:1014EC001C44FFF7EDFF401BA042FAD338BD00BFF0
:1014FC00080000240649CB6823F4E0631B041B0C92
:10150C00000200F4E0600343024A1A43CA607047C9
:10151C0000ED00E00000FA0530B4154BDB68C3F3B6
:10152C000223C3F10704042C28BF04241D1D062D1F
:10153C0014D9033B4FF0FF3505FA04F421EA0401FA
:10154C00994005FA03F322EA03031943002807DB49
:10155C000901C9B2074B195430BC70470023E9E7A5
:10156C0000F00F000901C9B2034B1954F4E700BF96
:10157C0000ED00E000E400E014ED00E0002807DBE3
:10158C0000F01F02400901239340024A42F8203028
:10159C00704700BF00E100E000280CDB00F01F02E8
:1015AC004009012393402030034A42F82030BFF316
:1015BC004F8FBFF36F8F704700E100E00138B0F13F
:1015CC00807F0AD2064B5860064AF02182F823101D
:1015DC000020986007221A6070470120704700BFF6
:1015EC0010E000E000ED00E070B50446FFF768FF86
:1015FC00002C00F09181054694F83530DBB2022BBB
:10160C0006D080236365002384F83430012070BD3C
:10161C0023688C498C4A934218BF8B4230D01832C5
:10162C0093422DD0183293422AD01832934227D0AD
:10163C001832934224D01832934221D0183293425C
:10164C001ED002F5567293421AD01832934217D01C
:10165C001832934214D01832934211D0183293425C
:10166C000ED0183293420BD01832934208D0183255
:10167C00934205D01A6822F00E021A60266809E01F
:10168C001A6822F01E021A602268536923F0800344
:10169C005361266823686B496B4A934218BF8B428F
:1016AC0042D0183293423FD0183293423CD0183279
:1016BC00934239D01832934236D01832934233D0F9
:1016CC001832934230D002F5567293422CD0183215
:1016DC00934229D01832934226D01832934223D009
:1016EC001832934220D0183293421DD018329342B4
:1016FC001AD01832934217D0544A934214D0143251
:10170C00934211D0143293420ED0143293420BD028
:10171C001432934208D01432934205D014329342BF
:10172C0002D01432934204D1226E136823F48073D6
:10173C00136023684349444A934218BF8B422FD00D
:10174C00183293422CD01832934229D0183293423B
:10175C0026D01832934223D01832934220D018321C
:10176C0093421DD002F55672934219D0183293420F
:10177C0016D01832934213D01832934210D018322C
:10178C0093420DD0183293420AD01832934207D0AC
:10179C001832934204D01A6822F001021A6003E056
:1017AC001A6822F001021A60336813F0010F0ED090
:1017BC00FFF786FE431B052BF6D920236365032315
:1017CC0084F83530002384F8343001201FE7236877
:1017DC001C491D4A934218BF8B4239D01832934290
:1017EC0036D01832934233D01832934230D018325C
:1017FC0093422DD0183293422AD01832934227D0DC
:10180C0002F55672934223D01832934220D01832EC
:10181C0093421DD0183293421AD01832934217D0EB
:10182C001832934214D01832934211D0183293428A
:10183C000ED0A16DE36D03F01F02012393404B60AA
:10184C000DE000BF1000024028000240085402586E
:10185C00A16DE36D03F01F023F2393408B6023685F
:10186C002E492F4A934218BF8B4242D018329342D2
:10187C003FD0183293423CD01832934239D01832B0
:10188C00934236D01832934233D01832934230D030
:10189C0002F5567293422CD01832934229D018324A
:1018AC00934226D01832934223D01832934220D040
:1018BC00183293421DD0183293421AD018329342E8
:1018CC0017D0184A934214D01432934211D01432C8
:1018DC0093420ED0143293420BD01432934208D060
:1018EC001432934205D01432934202D014329342F4
:1018FC000BD1636EA26E5A60E36E33B11A6822F498
:10190C0080721A60236F626F5A60012384F835303D
:10191C00002084F834007AE6012078E610000240BA
:10192C002800024008540258002800F0298108B50C
:10193C00024690F83530DBB2022B03D0802343658E
:10194C00012008BD0368904890498B4218BF834220
:10195C000CBF0121002166D03030834263D0183097
:10196C00834260D0183083425DD0183083425AD005
:10197C001830834257D01830834254D000F556703B
:10198C00834250D0183083424DD0183083424AD015
:10199C001830834247D01830834244D018308342E9
:1019AC0041D0183083423ED0183083423BD0196866
:1019BC0021F00E0119601368A0F5956073498B42F4
:1019CC0018BF83426AD072498B4267D018318B4260
:1019DC0064D018318B4261D018318B425ED01831F3
:1019EC008B425BD018318B4258D001F556718B422B
:1019FC0054D018318B4251D018318B424ED0183103
:101A0C008B424BD018318B4248D018318B4245D089
:101A1C0018318B4242D018318B423FD0196821F0DB
:101A2C00010119603EE0042082F8350081BB584A60
:101A3C0093422DD0183293422AD01832934227D099
:101A4C001832934224D01832934221D01832934248
:101A5C001ED002F5567293421AD01832934217D008
:101A6C001832934214D01832934211D01832934248
:101A7C000ED0183293420BD01832934208D0183241
:101A8C00934205D01A6822F001021A60002058E730
:101A9C001A6822F001021A60002052E7196821F03E
:101AAC00010119601368384838498B4218BF8342CA
:101ABC0042D018318B423FD018318B423CD0183178
:101ACC008B4239D018318B4236D018318B4233D0FF
:101ADC0018318B4230D001F556718B422CD0183115
:101AEC008B4229D018318B4226D018318B4223D00F
:101AFC0018318B4220D018318B421DD018318B42BB
:101B0C001AD018318B4217D022498B4214D0143181
:101B1C008B4211D014318B420ED014318B420BD02E
:101B2C0014318B4208D014318B4205D014318B42C6
:101B3C0002D014318B4217D1116E0B6823F48073D1
:101B4C000B60906DD36D03F01F0101238B4043603C
:101B5C00536E916E5960D36E33B1196821F4807154
:101B6C001960136F516F5960012382F835300023CF
:101B7C0082F83430136D2BB1104698470020E0E604
:101B8C00012070470020DCE61000024028000240D3
:101B9C00400002400854025830B4446B0268D2F83A
:101BAC008410704B194041EA8401C2F88410026819
:101BBC00D2F8841021F47F01856B41EA0541C2F80B
:101BCC008410826B22440468D4F88810194041EACE
:101BDC008201C4F888100468D4F8881021F4FE013E
:101BEC00C56B41EA0541C4F88810C16B02EB410298
:101BFC000468D4F8A010194041EA8201C4F8A0107E
:101C0C000468D4F8A01021F4FE01056C41EA0541EA
:101C1C00C4F8A010046C416C01FB04240268D2F8D7
:101C2C00B010194041EA8401C2F8B0100268D2F831
:101C3C00B01021F4FE01856C41EA0541C2F8B010E8
:101C4C00826CC16C01FB02440268D2F8AC101940E2
:101C5C0041EA8401C2F8AC10026D416D01FB0242F5
:101C6C000468D4F8F010194041EA8201C4F8F0106D
:101C7C000468D4F8F01021F47C11856D41EA05411B
:101C8C00C4F8F010816D02EB41020468D4F8C01066
:101C9C000B4043EA8202C4F8C0200268D2F8C0307C
:101CAC0023F47C13C16D43EA0143C2F8C0300268CF
:101CBC00D2F8C03023F07C53016E43EA0163C2F8C2
:101CCC00C030436B284A1A449200C266836B02EB05
:101CDC0083030367C16B03EBC1034367046C416C63
:101CEC0001FB04F103EB81038367846CC16C01FB82
:101CFC0004F103EB8103C367046D416D01FB04F137
:101D0C0003EB8103C0F88030816D03EBC103C0F895
:101D1C008430C46D856E05FB04F403EB8403C0F8BA
:101D2C008830016E01FB05F103EB8103C0F89030A4
:101D3C000E498B4207D8D0F8903093420ED900232D
:101D4C0042F8043BF7E7D0F89C3043F02003C0F88E
:101D5C009C30032380F89830012000E0002030BC38
:101D6C00704700BF0300FFFF002B0010FCD30040A6
:101D7C00F0B44C68002C30D10E698C6826430C688A
:101D8C0046EA84460D6ACC6944EA05648D692C43A5
:101D9C004D692C43CD6844EA0544D0F88470806EBC
:101DAC0003FB00F307EB830547F823606C600835F1
:101DBC000020CB680E4CE35C834216D91418E678ED
:101DCC00A3781B0443EA0663647843EA0423145C97
:101DDC00234345F8043B0430EBE70C698E6826433B
:101DEC000C68264346F08046CCE7F0BC704700BF39
:101DFC00405F000830B595B004464C22A04901A8BC
:101E0C00FEF776FE002C00F0388123689D4A934241
:101E1C0020D094F898300BB32268936923F0100308
:101E2C009361FFF74DFB054623689A6912F0080F82
:101E3C001AD0FFF745FB431B0A2BF5D9D4F89C307D
:101E4C0043F00103C4F89C30032384F8983001203C
:101E5C0015B030BD03F580736360DAE784F8993010
:101E6C002046FFF73FF8D7E79A6942F001029A61E2
:101E7C00FFF726FB054623689A6912F0010F0FD174
:101E8C00FFF71EFB401B0A28F5D9D4F89C3043F011
:101E9C000103C4F89C30032384F898300120D7E761
:101EAC009A6942F002029A61237C012B40D022688D
:101EBC00936943F040039361637C012B3ED022680D
:101ECC00936923F480439361A37C012B3CD022685B
:101EDC00936943F4805393612268936923F44073AC
:101EEC00A1680B4393612268936923F0A403936167
:101EFC002268136923F010031361E368012B29D0C6
:101F0C00002B2CD0022B00F09B802268936943F0AD
:101F1C00800393612268136943F010031361E36833
:101F2C00032B1CD12268936943F02003936116E0C4
:101F3C002268936923F040039361BDE7226893699B
:101F4C0043F480439361BFE72268936923F4805381
:101F5C009361C1E72268936943F004039361A36919
:101F6C005A1EE369013B1B0243EA4263226A013AAF
:101F7C0013436269013A216843EA0243CB61A368C7
:101F8C00B3F5407F62D0236E33B12268D2F8C030F3
:101F9C00616E0B43C2F8C030E36D226ED3420DD09C
:101FAC002168D1F8C83023F00703A26E14A800EB07
:101FBC00820252F84C2C1343C1F8C830236C6BB11D
:101FCC002168D1F8BC3023F00703626C14A800EB35
:101FDC00820252F84C2C1343C1F8BC30A36C73B181
:101FEC002168D1F8BC3023F07003E26C14A800EB2C
:101FFC00820252F84C2C43EA0213C1F8BC30236D18
:10200C0073B12168D1F8BC3023F4E063626D14A87D
:10201C0000EB820252F84C2C43EA0223C1F8BC308C
:10202C002268184B9A4222D00023C4F89430C4F88A
:10203C009C30012384F898302046FFF7ADFD07E76C
:10204C002268936943F02003936188E7A36A013BFC
:10205C00E26A013A43EA0223226B013A43EA021391
:10206C00626A013A216843EA0243CB608BE76268FB
:10207C00936823F003039360D6E70120E8E600BFE2
:10208C00E45E000800A0004090F89830013BDBB201
:10209C00012B07D9D0F89C3043F00203C0F89C30D8
:1020AC0001207047CB680A68D2B9072B0ED08A681A
:1020BC00DB0643EA82730A6943EA02434A69134323
:1020CC00C26E496842F82130002070470A69CB691A
:1020DC001B0243EA02438A69134343F06053EFE760
:1020EC0010B40A6942EA4372072B0DD08C684B6915
:1020FC0043EA8473006F496800EBC10440F8312057
:10210C006360002010BC70478B69F3E710B490F843
:10211C009840E4B2012C08D0D0F89C3043F0040372
:10212C00C0F89C30012010BC7047920042EA0112AA
:10213C0042EA4302036801990A43C3F88020002055
:10214C00F1E790F89830DBB2012B07D0D0F89C3037
:10215C0043F00403C0F89C300120704751B901686A
:10216C00D1F8F03023F07C5343EA0262C1F8F0203E
:10217C0000207047012909D00168D1F8B03023F054
:10218C00FE4343EA0262C1F8B020F1E70168D1F8DE
:10219C00A03023F0FE4343EA0262C1F8A020E7E737
:1021AC0090F89830DBB2012B07D0D0F89C3043F07C
:1021BC000403C0F89C3001207047022380F898304B
:1021CC000268936923F0010393610023C0F89C30EB
:1021DC001846704790F89830DBB2022B3ED102685B
:1021EC00936943F00103936100230268916911F034
:1021FC00010F0ED1322B01D80133F6E7D0F89C3009
:10220C0043F00103C0F89C30032380F89830012080
:10221C007047936923F0100393610023026891695E
:10222C0011F0080F0ED0322B01D80133F6E7D0F89D
:10223C009C3043F00103C0F89C30032380F89830A5
:10224C0001207047936943F0020393610023C0F8A7
:10225C009430012280F8982018467047D0F89C30B2
:10226C0043F00803C0F89C300120704788B110B5CA
:10227C000446FFF7AFFF2268D36D23F00303D36549
:10228C002046FEF791FE0020C4F89C0084F89800CC
:10229C0010BD0120704738B5044690F89830DBB279
:1022AC00022B2BD10368D3F8C00010F07C5F0CD04C
:1022BC00D3F8C40010F4001F0FD0D4F89C3043F4B2
:1022CC000073C4F89C3001201FE0D4F89C3043F01C
:1022DC002003C4F89C30012017E0D3F8C450C5F398
:1022EC0004452B462046FFF743FD22680123AB40F3
:1022FC00C2F8D030C4F89430002006E0D0F89C30FE
:10230C0043F00803C0F89C30012038BDF0B490F8BD
:10231C009840E4B2022C40F0D88040290CD04129DE
:10232C003FD0046D8C4271D8D0F89C3043F0200320
:10233C00C0F89C300120CFE00468D4F8A05015F40C
:10234C00FE0F0CD0D4F8A45015F07F0F0FD1D0F89D
:10235C009C3043F48073C0F89C300120BCE0D0F872
:10236C009C3043F02003C0F89C300120B4E0D4F83A
:10237C00A450C5F3006C15F0807F06D0D4F8A050A3
:10238C005FEAD57C01D14FF0000CD4F8A440C4F323
:10239C000524A444446F456C0CFB05F504EB850443
:1023AC003CE00468D4F8B05015F4FE0F0CD0D4F80F
:1023BC00B45015F07F0F0FD1D0F89C3043F48073DC
:1023CC00C0F89C30012087E0D0F89C3043F020030B
:1023DC00C0F89C3001207FE0D4F8B450C5F3006CF9
:1023EC0015F0807F06D0D4F8B0505FEAD57C01D1CF
:1023FC004FF0000CD4F8B440C4F30524A444846F0B
:10240C00C56C0CFB05F504EB850407E0C46F456D4A
:10241C0001FB05F504EB85044FF0000C256805F075
:10242C0080455560002D2CD12568C5F38A45156073
:10243C00256805F000559560256805F00045156187
:10244C00A588D561E58805F00F05D560656805F4AC
:10245C0080155561656805F400159561E57905F001
:10246C007F0515626568ED0F556204F108050024BF
:10247C00D6681A4FBE5DA64208D92E5D1E55013492
:10248C00F6E7256825F060451560D1E740290AD0AC
:10249C0041290DD01F290FD80268012303FA01F13D
:1024AC00C2F8981002E00368C3F8A8C0002013E03B
:1024BC000368C3F8B8C0F9E701F01F0102680123F3
:1024CC0003FA01F1C2F89C10F0E7D0F89C3043F00D
:1024DC000803C0F89C300120F0BC7047405F000836
:1024EC0090F89830013BDBB2012B07D9D0F89C3027
:1024FC0043F00203C0F89C300120704710B403680D
:10250C009C6D0C4223D1DC6D44F00104DC6511F4AC
:10251C00007F05D00468D4F8E0301343C4F8E030F1
:10252C0011F4806F05D00468D4F8E4301A43C4F871
:10253C00E4200068436D0C4A0A40134343650B4A80
:10254C00536943EA91715161002010BC70479C6D36
:10255C0031EA040402D00324DC65D8E7DC6D44F0D6
:10256C000204DC65D3E700BFFFFFCF3F00A80040AB
:10257C007047704770477047704770477047704797
:10258C00704770477047704770477047704700003E
:10259C002DE9F04F83B00446B74B1A695B699B0772
:1025AC0003EA8273019303681A6D02F4704A5A6D40
:1025BC000AEA020A1A6D02F00F095A6D09EA0209B9
:1025CC001A6D02F0F0085A6D08EA02081E6D06F04A
:1025DC0071565A6D16401F6D07F060775A6D174093
:1025EC005D6DD3F850B015F4807F02D01BF4807F62
:1025FC0064D115F4806F02D01BF4806F67D1019BFE
:10260C00002B74D1BAF1000F7CD1B9F1000F40F05E
:10261C008580B8F1000F40F08D8015F4006F03D069
:10262C001BF4006F40F0928015F4007F03D01BF474
:10263C00007F40F0968015F4002F03D01BF4002F80
:10264C0040F09F8015F4803F03D01BF4803F40F096
:10265C00A38015F4802F03D01BF4802F40F0A780AB
:10266C0015F4003F0FD01BF4003F0CD023684FF43F
:10267C0000321A65804B00221A61D4F89C3043F06A
:10268C008003C4F89C30002F40F09C804EB123682E
:10269C001E65B20F784B1A61D4F89C301E43C4F8F7
:1026AC009C602268754B9A4200F09680D4F89C305E
:1026BC00002B40F0F88003B0BDE8F08F4FF480722F
:1026CC001A656D4B00221A61FFF75BFF91E72368D7
:1026DC00D3F8DC10D3F8E4204FF480601865664B17
:1026EC000020186111402046FFF747FF87E7236859
:1026FC0000221A6501998A0F5F4B1A612046FFF779
:10270C0037FF7FE72368C3F850A04FEA9A725A4B01
:10271C001A6151462046FFF72CFF76E72368C3F871
:10272C0050904FEA9972544B1A6149462046FEF775
:10273C008DFB6EE72368C3F850804FEA98724E4BBE
:10274C001A6141462046FFF715FF66E723684FF4F0
:10275C0000621A65484B00221A612046FFF70BFFF6
:10276C0062E72368D3F8D810D3F8E0204FF4007058
:10277C001865414B0020186111402046FFF7FCFE04
:10278C0059E723684FF400221A653B4B00221A616B
:10279C002046FFF7F3FE55E723684FF480321A65A5
:1027AC00354B00221A612046FFF7E9FE51E72368FA
:1027BC004FF480221A65304B00221A612046FFF735
:1027CC00DFFE4DE723681F65BA0F2B4B1A613946A4
:1027DC002046FEF745FB59E763689A6812F0030F31
:1027EC003FF464AF196A01F00F015A6A186A00F0DD
:1027FC003008586A08EA00081F6A07F4C077586A5C
:10280C0007401E6A06F4FC46586A06401D6A05F429
:10281C00F025586A0540D3F82490D3F820A0114035
:10282C001CD1B8F1000F1ED119F0400F02D01AF0D4
:10283C00400F25D187BB36B163681E62D4F89C303B
:10284C001E43C4F89C60002D3FF430AF63681D62DA
:10285C00D4F89C301D43C4F89C5027E719622046DD
:10286C00FFF791FEDDE76368C3F820804146204600
:10287C00FFF78AFED8E700BF00A8004000A0004088
:10288C006368D96BDA6B4020186202F03F02090CC6
:10289C002046FFF77AFECDE763681F623946204673
:1028AC00FFF774FEC7E72046FFF76CFE03E700BF97
:1028BC00F0B482B000235FE086685F000325BD4062
:1028CC0026EA0506CD68BD4035438560466826EA94
:1028DC0004064D68C5F300149C403443446059E031
:1028EC00DD08083550F8257003F00704A6000F2406
:1028FC00B44027EA04070C69B4403C4340F8254037
:10290C005CE0092400E00024B4403C4302355C4EFA
:10291C0046F825404FF0B0442568D44325EA02061A
:10292C004F6817F4801F01D042EA05064FF0B045FE
:10293C002E606E6804EA06054F6817F4001F01D07C
:10294C0042EA06054FF0B04675604E4D6D6804EADC
:10295C0005064F6817F4003F01D042EA0506494DC1
:10296C006E602D682C404E6816F4803F01D042EA10
:10297C000504444A146001330A6832FA03F47BD02C
:10298C0001249C402240F6D04D6805F00305013D22
:10299C00012D91D94C6804F00304032C09D0C568AF
:1029AC005E000324B44025EA04058C68B4402C4333
:1029BC00C4604C6804F00304022C91D005685E00DE
:1029CC000324B44025EA04054C6804F00304B44025
:1029DC002C4304604C6814F4403FCCD02A4CD4F8FF
:1029EC00F45045F00205C4F8F450D4F8F44004F067
:1029FC0002040194019C9D08AE1C214C54F82670D5
:102A0C0003F00304A6000F24B44027EA04071F4C6C
:102A1C00A0423FF478AF04F58064A0421ED004F5C8
:102A2C008064A0421CD004F58064A0421AD004F546
:102A3C008064A04218D004F58064A04216D004F53E
:102A4C008064A04214D004F58064A04212D004F536
:102A5C000064A0423FF455AF0A2455E7012453E724
:102A6C00022451E703244FE704244DE705244BE7E8
:102A7C00062449E7072447E702B0F0BC704700BFC3
:102A8C00000400588000005800440258000002580E
:102A9C00002390E0092600E0002606FA04F4AC427C
:102AAC006BD005685C00032606FA04F42543056028
:102ABC0023FA06F5083550F8256003F007074FEAAE
:102ACC00870C0F2707FA0CF726EA070640F8256053
:102ADC00C56825EA0405C560456825EA020242601E
:102AEC00826822EA04048460013331FA03F260D074
:102AFC0001229A4012EA010CF6D09F08BD1C334CFF
:102B0C0054F8255003F00304A4000F2606FA04FE23
:102B1C000EEA05052E4EB042BED006F58066B042D8
:102B2C001DD006F58066B0421BD006F58066B0421B
:102B3C0019D006F58066B04217D006F58066B04213
:102B4C0015D006F58066B04213D006F58066B0420B
:102B5C0011D006F50066B0429CD00A269DE70126EE
:102B6C009BE7022699E7032697E7042695E70526B7
:102B7C0093E7062691E707268FE7164C256825EA8A
:102B8C000C052560656825EA0C0565604FF0B044BE
:102B9C00656825EA0C056560256825EA0C05256045
:102BAC000A4DBC1C55F8246026EA0E0645F8246034
:102BBC0077E7F0BD013331FA03F206D001229A40D7
:102BCC0012EA010CF6D0F0B597E7704700040058F4
:102BDC0000000258800000580AB181617047090456
:102BEC0081617047134BDB6813F0040F07D1114B55
:102BFC00DB6803F0070383421AD00120704710B53D
:102C0C000C4AD36823F007031843D060FEF758FC36
:102C1C000446084B5B6813F4005F07D1FEF750FCC9
:102C2C00001BB0F57A7FF4D9012000E0002010BD24
:102C3C000020704700480258002800F0D78238B5B1
:102C4C000446036813F0010F25D0AA4A136903F058
:102C5C003803926A102B15D0182B0FD06368B3F57C
:102C6C00803F3FD0002B53D1A24B1A6822F4803204
:102C7C001A601A6822F480221A6038E002F003020B
:102C8C00022AEBD19B4B1B6813F4003F03D0636803
:102C9C00002B00F0AD82236813F0020F00F0888047
:102CAC00944A1369926A13F038035AD0182B55D0F2
:102CBC00E368002B00F0A9808E490A6822F0190203
:102CCC0013430B60FEF7FCFB05468A4B1B6813F0A5
:102CDC00040F40F09180FEF7F3FB401B0228F4D95F
:102CEC0003208CE2834A136843F4803313606368D7
:102CFC002BB3FEF7E5FB05467E4B1B6813F4003F38
:102D0C00C9D1FEF7DDFB401B6428F5D9032076E220
:102D1C00B3F5A02F09D0774B1A6822F480321A60D1
:102D2C001A6822F480221A60E1E7724B1A6842F4A6
:102D3C0080221A601A6842F480321A60D7E7FEF7D4
:102D4C00BFFB05466B4B1B6813F4003FA3D0FEF78B
:102D5C00B7FB401B6428F5D9032050E212F0030F97
:102D6C00A6D1644B1B6813F0040F03D0E368002B4F
:102D7C0000F040825F4A136823F01903E1680B43AB
:102D8C001360FEF79DFB05465A4B1B6813F0040FAE
:102D9C0006D1FEF795FB401B0228F5D903202EE245
:102DAC00544A536823F0FE43216943EA016353609C
:102DBC00236813F0100F51D04E4A136903F03803F7
:102DCC00926A082B39D0182B33D0E369002B68D0CA
:102DDC00484A136843F080031360FEF771FB054605
:102DEC00444B1B6813F4807F52D1FEF769FB401BE8
:102DFC000228F5D9032002E23E4A536823F0FE4331
:102E0C00216943EA01635360D2E73A4A136823F01D
:102E1C0001031360FEF754FB0546364B1B6813F099
:102E2C00040FC5D0FEF74CFB401B0228F5D903203C
:102E3C00E5E102F00302012AC7D12E4B1B6813F403
:102E4C00807F03D0E369802B40F0D681294AD36878
:102E5C0023F07C53216A43EA0163D360236813F0A7
:102E6C00080F49D0636983B3224A536F43F00103BF
:102E7C005367FEF725FB05461E4B5B6F13F0020FE5
:102E8C003AD1FEF71DFB401B0228F5D90320B6E111
:102E9C00184AD36823F07C53216A43EA0163D36058
:102EAC00DCE7144A136823F080031360FEF708FB79
:102EBC000546104B1B6813F4807FCFD0FEF700FB48
:102ECC00401B0228F5D9032099E10A4A536F23F0DD
:102EDC0001035367FEF7F4FA0546064B5B6F13F0DC
:102EEC00020F09D0FEF7ECFA401B0228F5D903209B
:102EFC0085E100BF00440258236813F0200F29D04D
:102F0C00A3699BB1A84A136843F480531360FEF77E
:102F1C00D7FA0546A44B1B6813F4005F1AD1FEF7D1
:102F2C00CFFA401B0228F5D9032068E19E4A1368AA
:102F3C0023F480531360FEF7C3FA05469A4B1B68C3
:102F4C0013F4005F06D0FEF7BBFA401B0228F5D93C
:102F5C00032054E1236813F0040F21D1636A002B82
:102F6C0000F04C81904A126902F03802182A00F0E5
:102F7C00EA80022B75D08C4A136823F0807313609F
:102F8C00FEF79EFA0446884B1B6813F0007F00F096
:102F9C00D880FEF795FA001B0228F4D903202EE105
:102FAC00824A136843F480731360FEF789FA05466E
:102FBC007E4B1B6813F4807F06D1FEF781FA401B11
:102FCC006428F5D903201AE1A368012B0AD00BBBA6
:102FDC00754B1A6F22F001021A671A6F22F0040265
:102FEC001A6704E0704A136F43F001031367A36878
:102FFC0033B3FEF765FA05466B4B1B6F13F0020FEC
:10300C00ACD1FEF75DFA401B41F288339842F3D9FC
:10301C000320F4E0052B09D0634B1A6F22F0010258
:10302C001A671A6F22F004021A67E0E75E4B1A6FF8
:10303C0042F004021A671A6F42F001021A67D6E7CF
:10304C00FEF73EFA0546584B1B6F13F0020F85D066
:10305C00FEF736FA401B41F288339842F3D903202D
:10306C00CDE0514A136823F080731360FEF728FA01
:10307C0005464D4B1B6813F0007F06D0FEF720FA77
:10308C00401B0228F5D90320B9E0474B996A484AFE
:10309C000A40A16AE06A41EA00110A439A62226B73
:1030AC00013AC2F30802616B0139490289B20A4341
:1030BC00A16B0139090401F4FE010A43E16B0139EA
:1030CC00090601F0FE410A431A63DA6A22F0010292
:1030DC00DA62596B374A0A40A16C42EAC1025A6360
:1030EC00DA6A22F00C02216C0A43DA62DA6A22F004
:1030FC000202616C0A43DA62DA6A42F48032DA6202
:10310C00DA6A42F40032DA62DA6A42F48022DA6273
:10311C00DA6A42F00102DA621A6842F080721A60CE
:10312C00FEF7CEF90446204B1B6813F0007F06D146
:10313C00FEF7C6F9001B0228F5D903205FE000203A
:10314C005DE000205BE018498A6A086B012B57D0C0
:10315C0002F00303A16A8B4254D1C2F30512E36A55
:10316C009A4251D1C0F30802236B013B9A424DD1D4
:10317C00C0F34622636B013B9A4249D1C0F306422D
:10318C00A36B013B9A4245D1C0F30660E36B013B54
:10319C00984241D1044B5B6BC3F3CC03A26C9A42B3
:1031AC000AD100202BE000BF00440258004802580E
:1031BC000CFCFFFF0700FFFF184AD36A23F0010342
:1031CC00D362FEF77DF90546FEF77AF9A842FBD0EB
:1031DC00124A516B124B0B40A16C43EAC10353636F
:1031EC00D36A43F00103D362002008E0012070474A
:1031FC00012004E0012002E0012000E0002038BDA5
:10320C000120FCE70120FAE70120F8E70120F6E7AE
:10321C000120F4E70120F2E70120F0E70044025816
:10322C000700FFFFF8B57E4B1B6903F03803102B2A
:10323C0000F0F280182B10D013B17A4C2046F8BD58
:10324C00774B1B6813F0200F00F0E880744B186864
:10325C00C0F3C100744CC440F0E7714B9D6A05F09B
:10326C0003059C6AC4F30514D86A00F001005B6B7B
:10327C00C3F3CC0300FB03F0FDF7F8F80646002C73
:10328C00DCD0012D76D0022D00F0A4800DB32046A9
:10329C00FDF7ECF801466548FDF7F4F90446604B80
:1032AC00186BC0F30800FDF7E1F805464FF06451C8
:1032BC003046FDF733F901462846FDF727F84FF065
:1032CC007E51FDF723F801462046FDF727F9044609
:1032DC0071E0534B1B6813F0200F29D0504F3B6803
:1032EC00C3F3C1035048D840FDF7C0F8054620464B
:1032FC00FDF7BCF801462846FDF7C4F90446386BC7
:10330C00C0F30800FDF7B2F805464FF064513046A3
:10331C00FDF704F901462846FCF7F8FF4FF07E5103
:10332C00FCF7F4FF01462046FDF7F8F8044642E0AE
:10333C002046FDF79BF801463D48FDF7A3F90446EE
:10334C00374B186BC0F30800FDF790F805464FF0AB
:10335C0064513046FDF7E2F801462846FCF7D6FFEB
:10336C004FF07E51FCF7D2FF01462046FDF7D6F810
:10337C00044620E02046FDF779F801462B48FDF77E
:10338C0081F90446264B186BC0F30800FDF76EF864
:10339C0005464FF064513046FDF7C0F8014628460B
:1033AC00FCF7B4FF4FF07E51FCF7B0FF014620460E
:1033BC00FDF7B4F804461A4B1B6BC3F34623581C99
:1033CC00FDF754F801462046FDF75CF9FDF7F6F9D8
:1033DC00044633E72046FDF749F801461548FDF74A
:1033EC0051F904460E4B186BC0F30800FDF73EF87C
:1033FC0005464FF064513046FDF790F801462846DB
:10340C00FCF784FF4FF07E51FCF780FF014620460D
:10341C00FDF784F80446CEE7074C0FE7024C0DE7A6
:10342C000044025800093D000090D0030024744A67
:10343C000024744C20BCBE4B40787D01002800F069
:10344C00328170B50D4604469B4B1B6803F00F038D
:10345C008B420BD2984A136823F00F030B43136073
:10346C00136803F00F038B4240F01F81236813F0A5
:10347C00040F0CD02269914B9B6903F070039A42A4
:10348C0005D98E498B6923F070031A438A6123682E
:10349C0013F0080F0CD06269884BDB6903F07003E2
:1034AC009A4205D98549CB6923F070031A43CA6146
:1034BC00236813F0100F0CD0A269804BDB6903F466
:1034CC00E0639A4205D97D49CB6923F4E0631A4342
:1034DC00CA61236813F0200F0CD0E269774B1B6A8A
:1034EC0003F070039A4205D974490B6A23F07003F8
:1034FC001A430A62236813F0020F0CD0E2686F4B78
:10350C009B6903F00F039A4205D96C498B6923F030
:10351C000F031A438A61236813F0010F41D0674AE5
:10352C00936923F47063A1680B4393616368022B66
:10353C000AD0032B27D0012B2CD0604A126812F032
:10354C00040F06D10120ADE0126812F4003F00F028
:10355C00AE805A490A6922F0070213430B61FDF74A
:10356C00AFFF0646554B1B6903F038036268B3EB9B
:10357C00C20F16D0FDF7A4FF801B41F2883398428E
:10358C00F0D903208EE04D4A126812F0007FE0D192
:10359C00012087E0494A126812F4807FD9D10120BA
:1035AC0080E0236813F0020F0CD0E268434B9B6958
:1035BC0003F00F039A4205D240498B6923F00F03A5
:1035CC001A438A613C4B1B6803F00F03AB420AD9C8
:1035DC00394A136823F00F032B431360136803F06D
:1035EC000F03AB4265D1236813F0040F0CD0226992
:1035FC00324B9B6903F070039A4205D22F498B69B9
:10360C0023F070031A438A61236813F0080F0CD05F
:10361C0062692A4BDB6903F070039A4205D2274991
:10362C00CB6923F070031A43CA61236813F0100F9F
:10363C000CD0A269214BDB6903F4E0639A4205D2FA
:10364C001E49CB6923F4E0631A43CA61236813F063
:10365C00200F0CD0E269194B1B6A03F070039A42DD
:10366C0005D216490B6A23F070031A430A62FFF75E
:10367C00D9FD12498B69C3F30323114AD35C03F0C0
:10368C001F03D8408B6903F00F03D35C03F01F03B7
:10369C0020FA03F30B4A13600B4B18600B4B1868A2
:1036AC00FDF7ACFE70BD012070470120FAE7012048
:1036BC00F8E70120F6E700BF002000520044025852
:1036CC00305F000804000024000000240C000024DB
:1036DC0008B5FFF7A7FD0B4A9369C3F303230A4907
:1036EC00CB5C03F01F0320FA03F3926902F00F0284
:1036FC00885C00F01F0023FA00F0044A1060044AB2
:10370C00136008BD00440258305F00080400002418
:10371C000000002408B5FFF7DBFF054BDB69C3F3A2
:10372C000213044AD35C03F01F03D84008BD00BF4A
:10373C0000440258305F000808B5FFF7C9FF054B7D
:10374C00DB69C3F30223044AD35C03F01F03D840A4
:10375C0008BD00BF00440258305F0008404B9B6A14
:10376C0003F00303032B79D070B505460E463C4A93
:10377C00136823F080631360FDF7A2FE0446384BF8
:10378C001B6813F0006F06D0FDF79AFE031B022B8B
:10379C00F5D9032070BD324B9A6A22F47C32296829
:1037AC0042EA01329A626A68013AC2F30802A968D5
:1037BC000139490289B20A43E9680139090401F463
:1037CC00FE010A4329690139090601F0FE410A4349
:1037DC009A63DA6A22F0C00269690A43DA62DA6A29
:1037EC0022F02002A9690A43DA62DA6A22F0100296
:1037FC00DA62D96B1B4A0A40E96942EAC102DA6310
:10380C00DA6A42F01002DA62C6B91A46DB6A43F48D
:10381C000023D362124A136843F080631360FDF7F0
:10382C004FFE04460E4B1B6813F0006F14D1FDF7CE
:10383C0047FE001B0228F5D90320ABE7012E05D06B
:10384C00074AD36A43F40013D362E3E7044AD36A0A
:10385C0043F48013D362DDE700209BE7012070471F
:10386C00004402580700FFFF404B9B6A03F0030320
:10387C00032B79D070B505460E463C4A136823F0ED
:10388C0080531360FDF71CFE0446384B1B6813F085
:10389C00005F06D0FDF714FE031B022BF5D90320A5
:1038AC0070BD324B9A6A22F07C72296842EA01524E
:1038BC009A626A68013AC2F30802A968013949029E
:1038CC0089B20A43E9680139090401F4FE010A438B
:1038DC0029690139090601F0FE410A431A64DA6AC2
:1038EC0022F4406269690A43DA62DA6A22F40072ED
:1038FC00A9690A43DA62DA6A22F48072DA62596CD4
:10390C001B4A0A40E96942EAC1025A64DA6A42F483
:10391C008072DA62C6B91A46DB6A43F48003D3625A
:10392C00124A136843F080531360FDF7C9FD044637
:10393C000E4B1B6813F0005F14D1FDF7C1FD001B8B
:10394C000228F5D90320ABE7012E05D0074AD36A2C
:10395C0043F08073D362E3E7044AD36A43F4000371
:10396C00D362DDE700209BE701207047004402583A
:10397C000700FFFFF8B50446016801F00062002360
:10398C00134330D0436EB3F5001F26D00ED8EBB1E5
:10399C00B3F5801F07D102210830FFF7DFFE054683
:1039AC0045B12E4621E0012635461EE0B3F5401FF9
:1039BC0009D10025A84A136D23F44013616E0B4303
:1039CC001365002611E0012635460EE0A24AD36AA3
:1039DC0043F40033D3620025ECE702212830FFF7D3
:1039EC0043FF0546DCE700263546216801F480726A
:1039FC000023134314D0A36D042B37D8DFE803F056
:103A0C0003282F080800944AD36A43F40033D36286
:103A1C007DBB914A136D23F00703A16D0B43136516
:103A2C00216801F480620023134336D0D4F8A4300B
:103A3C00B3F5800F55D021D8002B4CD0B3F5001F17
:103A4C0019D1002104F10800FFF788FE05461BE0A0
:103A5C00002104F10800FFF781FE0546D8E700219C
:103A6C0004F12800FFF700FF0546D1E70126354693
:103A7C00D6E72E46D4E7012635460EE0B3F5000F07
:103A8C0002D0B3F5200F20D195BB734A936D23F46C
:103A9C006003D4F8A4100B439365216801F4006211
:103AAC000023134339D0D4F8A830B3F1007F5CD095
:103ABC0023D8002B53D0B3F1807F1BD1002104F10C
:103ACC000800FFF74BFE05461DE0B3F5C00FDBD039
:103ADC0001263546E1E7604AD36A43F40033D362EA
:103AEC00D2E7002104F12800FFF7BEFE0546CBE724
:103AFC002E46D2E7012635460FE0B3F1806F02D097
:103B0C00B3F1A06F25D1002D36D1534A936D23F01C
:103B1C00E063D4F8A8100B439365216801F00072A0
:103B2C000023134331D0E36C202B45D029D833B17B
:103B3C00102B23D1484AD36A43F40033D362002DAF
:103B4C0041D1454AD36C23F03003E16C0B43D36471
:103B5C001BE0B3F1407FD6D001263546DDE73E4A67
:103B6C00D36A43F40033D362CDE7002104F128007B
:103B7C00FFF77AFE0546C6E72E46CEE70126354608
:103B8C0003E0302BDBD001263546216801F480524E
:103B9C00002313432BD0E36DB3F5005F4FD017D840
:103BAC00002B46D0B3F5805F0FD1002104F1080043
:103BBC00FFF7D4FD054611E0022104F10800FFF7E0
:103BCC00CDFD0546BBE72E46DFE7012635460EE068
:103BDC00B3F5405F02D0B3F5804F27D1002D35D11E
:103BEC001D4A136D23F4E043E16D0B43136521680B
:103BFC0001F40052002313433BD0236EB3F5003F76
:103C0C0058D02BD843B1B3F5803F21D1012104F119
:103C1C000800FFF7A3FD0546002D52D10E4A136D87
:103C2C0023F4E023216E0B43136522E00126354675
:103C3C00DDE7094AD36A43F40033D362CEE70021AF
:103C4C0004F12800FFF710FE0546C7E72E46CEE725
:103C5C00012635460DE000BF00440258B3F5802F15
:103C6C00DAD0B3F5A02FD7D0B3F5403FD4D001268E
:103C7C003546216801F480420023134331D0D4F837
:103C8C00AC30B3F1005F49D020D843B1B3F1805FC1
:103C9C0019D1012104F10800FFF760FD0546002D44
:103CAC0043D1954A936D23F0E043D4F8AC100B4309
:103CBC00936516E0012104F12800FFF7D5FD0546B8
:103CCC00AAE72E46D5E7012635460AE0B3F1804F28
:103CDC00E5D0B3F1A04FE2D0B3F1405FDFD00126C5
:103CEC003546216801F400420023134309D0E36EEA
:103CFC00B3F1805F1BD0B3F1005F26D0E3B1012696
:103D0C003546216801F08072002313433FD0A36C29
:103D1C00032B38D8DFE803F027223027012104F1E8
:103D2C002800FFF7A1FD0546B9E72E46D9E7724AF0
:103D3C00D36A43F40033D36275B96F4A136D23F021
:103D4C004053E16E0B431365DBE7012104F10800DE
:103D5C00FFF704FD0546EFE72E46D2E7664AD36A25
:103D6C0043F40033D3628DB9634AD36C23F003035D
:103D7C00A16C0B43D3640AE0022104F10800FFF7A5
:103D8C00EDFC0546EFE70126354600E02E4621689E
:103D9C0001F480020023134321D1216801F00102B8
:103DAC000023134300F09780A36F282B00F291801F
:103DBC00DFE803F07F8F8F8F8F8F8F8F798F8F8FAF
:103DCC008F8F8F8F888F8F8F8F8F8F8F7F8F8F8F0E
:103DDC008F8F8F8F7F8F8F8F8F8F8F8F7F00474A23
:103DEC00136843F480731360FDF76AFB0746434B7B
:103DFC001B6813F4807F05D1FDF762FBC01B6428A0
:103E0C00F5D90325002D4AD13B4B1B6FD4F8B020BC
:103E1C00534013F4407F0CD0374B1A6F22F440728E
:103E2C00196F41F480311967196F21F480311967CA
:103E3C001A67D4F8B030B3F5807F15D08DBBD4F8A9
:103E4C00B03003F44072B2F5407F1ED02A4A136999
:103E5C0023F47C53136128490B6FD4F8B020C2F3C0
:103E6C000B0213430B6798E7FDF72AFB0746224B1F
:103E7C001B6F13F0020FE1D1FDF722FBC01B41F2C7
:103E8C0088339842F3D90325D8E71B48026922F4FA
:103E9C007C521B4901EA131313430361DBE72E46E3
:103EAC007BE72E4679E7012104F10800FFF756FC69
:103EBC000546F5B9104A536D23F03803A16F0B4337
:103ECC00536508E0012104F12800FFF7CDFC0546FD
:103EDC00EFE701263546216801F002020023134367
:103EEC002AD0636F052B23D8DFE803F0120C1B12CA
:103EFC0012122E46EFE700BF004402580048025849
:103F0C00CFFFFF00012104F10800FFF727FC054655
:103F1C008DB9B54A536D23F00703616F0B4353659D
:103F2C000AE0012104F12800FFF79EFC0546EFE7AB
:103F3C000126354600E02E46216801F004020023DC
:103F4C00134323D0D4F89030052B1BD8DFE803F0B3
:103F5C00090313090909012104F10800FFF7FEFB0D
:103F6C00054695B9A04A936D23F00703D4F8901039
:103F7C000B4393650AE0012104F12800FFF774FC60
:103F8C000546EEE70126354600E02E46216801F095
:103F9C0020020023134328D0D4F88C30B3F1005FF7
:103FAC0044D017D843B1B3F1805F10D1002104F194
:103FBC000800FFF7D3FB0546002D3ED18A4A536D0E
:103FCC0023F0E043D4F88C100B4353650DE001262D
:103FDC0035460AE0B3F1804FEED0B3F1A04FEBD0F1
:103FEC00B3F1405FE8D001263546216801F040026C
:103FFC000023134331D0D4F89830B3F5006F4FD071
:10400C0020D843B1B3F5806F19D1002104F1080019
:10401C00FFF7A4FB0546002D49D1734A936D23F499
:10402C00E053D4F898100B43936516E0022104F189
:10403C002800FFF719FC0546BEE72E46D5E70126FA
:10404C0035460AE0B3F5805FE5D0B3F5A05FE2D06A
:10405C00B3F5406FDFD001263546216801F08002B0
:10406C000023134333D0D4F89C30B3F5804F00F0C9
:10407C00B28021D843B1B3F5005F1AD1002104F10D
:10408C000800FFF76BFB0546002D40F0AB80564A4D
:10409C00936D23F46043D4F89C100B43936516E0A6
:1040AC00022104F12800FFF7DFFB0546B3E72E469B
:1040BC00D3E7012635460AE0B3F5004FE4D0B3F55B
:1040CC00204FE1D0B3F5C04FDED001263546216834
:1040DC0001F00802002313430DD0D4F88030B3F55F
:1040EC00805F00F08380404A536D23F44053D4F832
:1040FC0080100B435365216801F010020023134319
:10410C000CD0D4F89430B3F5807F79D0364A936DC7
:10411C0023F44073D4F894100B439365216801F495
:10412C000022002313430CD0D4F8A030B3F5803F09
:10413C0000F08080B3F5003F72D0002B6AD00126CE
:10414C003546216801F48022002313430DD0D4F8A6
:10415C008430B3F5001F00F08580B3F5401F77D095
:10416C00B3F5801F6FD001263546216801F48032EB
:10417C000023134308D0236D002B7CD0B3F5803F74
:10418C0000F0878001263546216801F0005200239B
:10419C00134340F08780216801F40032002313435D
:1041AC0000F08D80E36FB3F5807F00F0F78040F274
:1041BC008380B3F5007F03D0B3F5407F40F0EC80F3
:1041CC00002D40F0F180084A536D23F44073E16FE9
:1041DC000B43536573E0022104F12800FFF744FB05
:1041EC00054651E72E4672E700440258022104F1BD
:1041FC002800FFF739FB00283FF475AF012672E762
:10420C00022104F12800FFF72FFB00283FF47EAFBA
:10421C0001267BE7002104F10800FFF79FFA054611
:10422C007DB97D4A936D23F44033D4F8A0100B4331
:10423C00936586E7022104F12800FFF715FB05467C
:10424C00EEE72E467DE7744AD36A43F40033D3621B
:10425C007DB9714A536D23F44013D4F884100B4389
:10426C00536582E7012104F12800FFF7FDFA0546AA
:10427C00EEE72E4679E7684AD36A43F40033D362FB
:10428C0075B9654AD36C23F48033216D0B43D36429
:10429C007AE7022104F10800FFF760FA0546EFE720
:1042AC002E4671E7022104F12800FFF7DDFA002801
:1042BC003FF471AF01266EE7002B81D001262168F7
:1042CC0001F480120023134306D0534A136D23F0DC
:1042DC000043216F0B431365216801F40012002386
:1042EC00134306D04C4A136D23F08073A16E0B431D
:1042FC001365216801F080420023134309D0464B1B
:10430C001A6922F400421A611A69D4F8B4100A43EB
:10431C001A61216801F000420023134306D03E4A83
:10432C00D36C23F04053616D0B43D364216801F4CB
:10433C0000020023134307D0374A536D23F4400384
:10434C00D4F888100B4353656168002201F0010317
:10435C0013432BD16168002201F0020313432ED1C9
:10436C006168002201F00403134331D1616800221B
:10437C0001F00803134334D16168002201F01003EB
:10438C00134337D16168002201F0200313433AD163
:10439C0006B101263046F8BD012690E71E4AD36AC5
:1043AC0043F40033D3620BE72E4688E7002104F177
:1043BC000800FFF7D3F90028CCD00646CAE7012144
:1043CC0004F10800FFF7CAF90028C9D00646C7E770
:1043DC00022104F10800FFF7C1F90028C6D00646F7
:1043EC00C4E7002104F12800FFF73EFA0028C3D0EF
:1043FC000646C1E7012104F12800FFF735FA002831
:10440C00C0D00646BEE7022104F12800FFF72CFAC3
:10441C000028BDD00646BBE70044025808B5FFF79C
:10442C0057F9054B1B6AC3F30213044AD35C03F020
:10443C001F03D84008BD00BF00440258305F00087D
:10444C002DE9F0410446864B9D6A9E6AC6F30536FB
:10445C00D86AC0F30010DB6BC3F3CC0300FB03F092
:10446C00FCF704F8002E00F0F58005F00305074674
:10447C00012D79D0022D00F0CB800DB33046FBF727
:10448C00F5FF01467748FCF7FDF80546744B986B31
:10449C00C0F30800FBF7EAFF06464FF064513846BC
:1044AC00FCF73CF801463046FBF730FF4FF07E51ED
:1044BC00FBF72CFF01462846FCF730F8054674E064
:1044CC00674B1B6813F0200F2CD0DFF89481D8F8C1
:1044DC000030C3F3C1036448D840FBF7C7FF05465F
:1044EC003046FBF7C3FF01462846FCF7CBF80546E0
:1044FC00D8F83800C0F30800FBF7B8FF06464FF0B9
:10450C0064513846FCF70AF801463046FBF7FEFECC
:10451C004FF07E51FBF7FAFE01462846FBF7FEFFF3
:10452C00054642E03046FBF7A1FF01464F48FCF739
:10453C00A9F805464A4B986BC0F30800FBF796FFA9
:10454C0006464FF064513846FBF7E8FF014630460B
:10455C00FBF7DCFE4FF07E51FBF7D8FE01462846F8
:10456C00FBF7DCFF054620E03046FBF77FFF0146FA
:10457C003C48FCF787F80546394B986BC0F30800AC
:10458C00FBF774FF06464FF064513846FBF7C6FF45
:10459C0001463046FBF7BAFE4FF07E51FBF7B6FEF4
:1045AC0001462846FBF7BAFF05462D4EB06BC0F30B
:1045BC004620FBF75BFF4FF07E51FBF7A7FE014651
:1045CC002846FCF75FF8FCF7F9F82060B06BC0F3F5
:1045DC000640FBF74BFF4FF07E51FBF797FE014671
:1045EC002846FCF74FF8FCF7E9F86060B06BC0F3B5
:1045FC000660FBF73BFF4FF07E51FBF787FE014651
:10460C002846FCF73FF8FCF7D9F8A060BDE8F0812C
:10461C003046FBF72BFF01461548FCF733F80546EF
:10462C000F4B986BC0F30800FBF720FF06464FF0CA
:10463C0064513846FBF772FF01463046FBF766FEC5
:10464C004FF07E51FBF762FE01462846FBF766FFF2
:10465C000546AAE7002323606360A360D6E700BF8A
:10466C00004402580024744A0090D0030024744C77
:10467C0020BCBE4B2DE9F0410446864B9D6A9E6AD8
:10468C00C6F30556D86AC0F300205B6CC3F3CC03A9
:10469C0000FB03F0FBF7EAFE002E00F0F58005F0BE
:1046AC0003050746012D79D0022D00F0CB800DB308
:1046BC003046FBF7DBFE01467748FBF7E3FF054688
:1046CC00744B186CC0F30800FBF7D0FE06464FF095
:1046DC0064513846FBF722FF01463046FBF716FEC5
:1046EC004FF07E51FBF712FE01462846FBF716FFF2
:1046FC00054674E0674B1B6813F0200F2CD0DFF8D5
:10470C009481D8F80030C3F3C1036448D840FBF758
:10471C00ADFE05463046FBF7A9FE01462846FBF7E1
:10472C00B1FF0546D8F84000C0F30800FBF79EFE29
:10473C0006464FF064513846FBF7F0FE0146304612
:10474C00FBF7E4FD4FF07E51FBF7E0FD01462846F8
:10475C00FBF7E4FE054642E03046FBF787FE0146D8
:10476C004F48FBF78FFF05464A4B186CC0F3080007
:10477C00FBF77CFE06464FF064513846FBF7CEFE45
:10478C0001463046FBF7C2FD4FF07E51FBF7BEFDF4
:10479C0001462846FBF7C2FE054620E03046FBF7F3
:1047AC0065FE01463C48FBF76DFF0546394B186C1E
:1047BC00C0F30800FBF75AFE06464FF0645138462A
:1047CC00FBF7ACFE01463046FBF7A0FD4FF07E51E7
:1047DC00FBF79CFD01462846FBF7A0FE05462D4E37
:1047EC00306CC0F34620FBF741FE4FF07E51FBF7D7
:1047FC008DFD01462846FBF745FFFBF7DFFF2060E8
:10480C00306CC0F30640FBF731FE4FF07E51FBF7E6
:10481C007DFD01462846FBF735FFFBF7CFFF6060B7
:10482C00306CC0F30660FBF721FE4FF07E51FBF7B6
:10483C006DFD01462846FBF725FFFBF7BFFFA06087
:10484C00BDE8F0813046FBF711FE01461548FBF739
:10485C0019FF05460F4B186CC0F30800FBF706FE5A
:10486C0006464FF064513846FBF758FE0146304679
:10487C00FBF74CFD4FF07E51FBF748FD01462846F7
:10488C00FBF74CFE0546AAE7002323606360A36098
:10489C00D6E700BF004402580024744A0090D003AD
:1048AC000024744C20BCBE4B026852E8003F23F439
:1048BC00907342E800310029F6D1026802F1080336
:1048CC0053E8001F0D4B0B40083242E80031002921
:1048DC00F3D1C36E012B06D02023C0F88C300023FB
:1048EC00C36643677047026852E8003F23F0100329
:1048FC0042E800310029F6D1EEE700BFFEFFFFEFE2
:10490C00704708B5026852E8003F23F0400342E8C4
:10491C0000310029F6D12023C0F8883000238367AA
:10492C00FFF7EEFF08BD704708B5806B0023A0F8B9
:10493C005E30A0F85630FFF7F6FF08BD7047000058
:10494C0070B504460168CB6908688D6840F60F02A3
:10495C001A4008D113F0200F05D010F0200F34D1DD
:10496C0015F0805F31D12AB1B34A2A4033D1B34E0E
:10497C00304230D1E26E012A00F0C68013F4801F61
:10498C0003D015F4800F40F09B8113F0800F07D0FB
:10499C0010F0800F40F09B8115F4000F40F09781D0
:1049AC0013F0400F03D010F0400F40F0978113F438
:1049BC00000F03D010F0804F40F0948113F0807FF3
:1049CC0002D00028C0F2928170BD636F002BFBD027
:1049DC0020469847F8E713F0010F09D010F4807FB8
:1049EC0006D001260E62D4F890103143C4F8901012
:1049FC0013F0020F0BD015F0010F08D0216802261E
:104A0C000E62D4F8901041F00401C4F8901013F029
:104A1C00040F0BD015F0010F08D0216804260E628C
:104A2C00D4F8901041F00201C4F8901013F0080F64
:104A3C000BD010F0200F00D13AB12268082111627E
:104A4C00D4F890200A43C4F8902013F4006F0CD0D3
:104A5C0010F0806F09D022684FF400611162D4F815
:104A6C00902042F02002C4F89020D4F89020002A24
:104A7C00AAD013F0200F09D010F0200F02D115F09E
:104A8C00805F03D0636F0BB120469847D4F8902019
:104A9C0023689B6813F0400F02D112F0280F2CD022
:104AAC002046FFF701FF23689B6813F0400F20D0CE
:104ABC00226802F1080353E8003F23F04003083258
:104ACC0042E800310029F3D1D4F880306BB15C4A54
:104ADC001A65D4F88000FCF727FF00283FF474AF68
:104AEC00D4F88000036D98476EE72046FFF71BFF54
:104AFC006AE72046FFF717FF66E72046FFF713FF2C
:104B0C000023C4F890305FE713F0100F3FF436AF7A
:104B1C0010F0100F3FF432AF10230B6223689B6828
:104B2C0013F0400F00F09280D4F8802013684548B1
:104B3C0045498B4218BF83422DD018318B422AD065
:104B4C0018318B4227D018318B4224D018318B422C
:104B5C0021D018318B421ED018318B421BD001F55D
:104B6C0056718B4217D018318B4214D018318B42AE
:104B7C0011D018318B420ED018318B420BD018311A
:104B8C008B4208D018318B4205D018318B4202D0A1
:104B9C005B689BB201E05B689BB2002B3FF414AFE7
:104BAC00B4F85C1099427FF60FAFA4F85E30D3696D
:104BBC00B3F5807F32D0226852E8003F23F4807333
:104BCC0042E800310029F6D1226802F1080353E8CB
:104BDC00003F23F00103083242E800310029F3D1F1
:104BEC00226802F1080353E8003F23F04003083227
:104BFC0042E800310029F3D12023C4F88C30002383
:104C0C00E366226852E8003F23F0100342E80031CB
:104C1C000029F6D1D4F88000FCF7E6FC02232367C8
:104C2C00B4F85C10B4F85E309BB2C91A89B2204655
:104C3C00FFF784FEC8E600BF01000010200100044D
:104C4C00354900081000024028000240B4F85C10FE
:104C5C00B4F85E309BB2C91A89B2B4F85E309BB21C
:104C6C00002B3FF4B1AE00293FF4AEAE226852E8FF
:104C7C00003F23F4907342E800300028F6D12268FC
:104C8C0002F1080353E8000F1A4B0340083242E8C4
:104C9C0000300028F3D12023C4F88C300023E366C5
:104CAC006367226852E8003F23F0100342E80030AB
:104CBC000028F6D1022323672046FFF73FFE83E648
:104CCC004FF480130B62204600F0F0FC7CE6A36FDF
:104CDC00002B3FF479AE2046984775E62046FFF747
:104CEC0010FE71E6204600F0E3FC6DE6204600F075
:104CFC00DEFC69E6FEFFFFEF2DE9F04186B00446CD
:104D0C00016883680269134342691343C269134300
:104D1C000868914A024013430B602268536823F4DD
:104D2C004053E1680B435360A16922688B4B9A4254
:104D3C0001D0236A19439068894B03400B4393605D
:104D4C002268D36A23F00F03616A0B43D362226893
:104D5C00844B9A4229D0844B9A4200F09480834B26
:104D6C009A4200F0AA80824B9A4200F0C080814B9C
:104D7C009A4200F0D680804B9A4200F009817F4B1A
:104D8C009A4200F02E817E4B9A4200F041817D4B7D
:104D9C009A4200F054817C4B9A4200F079816F4B1F
:104DAC009A4200F09E81802333E0784B5B6D03F0D8
:104DBC003803282B65D8DFE813F029006400640061
:104DCC0064006400640064006400AC01640064006E
:104DDC00640064006400640064002B0064006400E0
:104DEC00640064006400640064005E00640064009D
:104DFC00640064006400640064006000640064008B
:104E0C00640064006400640064006200012300E03C
:104E1C00082352498A4200F09581E069B0F5004FB1
:104E2C0000F00D82202B00F26682202B00F2BA8259
:104E3C00DFE813F087028D02B802B8029002B802C4
:104E4C00B802B8029502B802B802B802B802B802A9
:104E5C00B802B8029A02B802B802B802B802B80294
:104E6C00B802B802B802B802B802B802B802B80266
:104E7C00B802B802A6021023CBE72023C9E74023CF
:104E8C00C7E78023C5E7414B5B6D03F00703052B98
:104E9C0011D8DFE813F00600400108000A000C00EE
:104EAC000E000023B5E70823B3E71023B1E7202356
:104EBC00AFE74023ADE78023ABE7344B5B6D03F0EA
:104ECC000703052B11D8DFE813F0060028010800B2
:104EDC000A000C000E0000239BE7082399E710231F
:104EEC0097E7202395E7402393E7802391E7274B0F
:104EFC005B6D03F00703052B11D8DFE813F00600F8
:104F0C00100108000A000C000E00002381E70823A2
:104F1C007FE710237DE720237BE7402379E780237D
:104F2C0077E71A4B5B6D03F00703052B11D8DFE80D
:104F3C0013F00600F80008000A000C000E00002315
:104F4C0067E7082365E7102363E7202361E7402325
:104F5C005FE780235DE700BFF369FFCF000C0058CB
:104F6C00FFF4FF11001001400044004000480040D5
:104F7C00004C0040005000400014014000780040FC
:104F8C00007C004000180140001C01400044025805
:104F9C00694B5B6D03F03803282B20D8DFE803F056
:104FAC00151F1F1F1F1F1F1FC31F1F1F1F1F1F1F6B
:104FBC00171F1F1F1F1F1F1F191F1F1F1F1F1F1F03
:104FCC001B1F1F1F1F1F1F1F1D00012321E708236D
:104FDC001FE710231DE720231BE7402319E780233D
:104FEC0017E7554B5B6D03F00703052B0ED8DFE875
:104FFC0003F0039C0507090B00230AE7082308E7C5
:10500C00102306E7202304E7402302E7802300E770
:10501C00494B5B6D03F00703052B0ED8DFE803F05B
:10502C0003870507090B0023F3E60823F1E6102399
:10503C00EFE62023EDE64023EBE68023E9E63E4B4A
:10504C005B6D03F03803282B20D8DFE803F0151F25
:10505C001F1F1F1F1F1F721F1F1F1F1F1F1F171F09
:10506C001F1F1F1F1F1F191F1F1F1F1F1F1F1B1F4E
:10507C001F1F1F1F1F1F1D000123CAE60823C8E6A0
:10508C001023C6E62023C4E64023C2E68023C0E6F4
:10509C00294B5B6D03F03803282B20D8DFE803F095
:1050AC00151F1F1F1F1F1F1F4E1F1F1F1F1F1F1FDF
:1050BC00171F1F1F1F1F1F1F191F1F1F1F1F1F1F02
:1050CC001B1F1F1F1F1F1F1F1D000123A1E60823ED
:1050DC009FE610239DE620239BE6402399E6802340
:1050EC0097E603F50E339B6D03F00703052B0ED8E3
:1050FC00DFE803F003260507090B022389E60823E2
:10510C0087E6102385E6202383E6402381E680236F
:10511C007FE604237DE604237BE6042379E604235F
:10512C0077E6042375E6042373E6042371E604236F
:10513C006FE604236DE600BF00440258042368E6C2
:10514C00042366E6202B27D8022BC0F01D81023BDE
:10515C001E2B00F21B81DFE813F0520019015800DE
:10516C001901190119015D00190119011901190120
:10517C00190119011901620019011901190119010B
:10518C001901190119011901190119011901190143
:10519C001901190119016E00402B2ED14FF400405A
:1051AC00626A824B33F81220B0FBF2F3656805EBB0
:1051BC004501994200F2EC80B3EB053F00F2EA8026
:1051CC004FF0000892B200234146FBF717FB0F0289
:1051DC0047EA1067060268082A464346301847F12A
:1051EC000001FBF70BFBA0F54072714B9A4200F2E9
:1051FC00D3802368D860404698E0012096E0FFF702
:10520C000DF90028CCD1002090E003A8FFF718F985
:10521C000498F6E76846FFF72DFA0198F1E7654B1D
:10522C001B6813F0200F08D0624B1B68C3F3C1033B
:10523C006148D840E5E76148B2E75F48B0E7202B0A
:10524C0015D8202B00F2AA80DFE803F03238A8A88A
:10525C003BA8A8A840A8A8A8A8A8A8A845A8A8A8FA
:10526C00A8A8A8A8A8A8A8A8A8A8A8A85100402B96
:10527C001CD1626A4D4B33F81230B0FBF3F062680C
:10528C00530803EB4000B0FBF2F0A0F110024FF614
:10529C00EF739A4200F2848083B223F00F03C0F3C1
:1052AC00420018432368D86000203FE001203DE015
:1052BC00FEF730FA0028DCD1002037E0FEF73CFA8C
:1052CC00F8E703A8FFF7BCF80498F3E76846FFF784
:1052DC00D1F90198EEE7374B1B6813F0200F08D07B
:1052EC00344B1B68C3F3C1033348D840E2E733485F
:1052FC00BFE73148BDE7402B17D14FF40040626A3D
:10530C002A4B33F81230B0FBF3F0636800EB530018
:10531C00B0FBF3F0A0F110024FF6EF739A4243D8B2
:10532C00236880B2D860002000E001200123A4F89B
:10533C006A30A4F8683000236367A36706B0BDE841
:10534C00F081FEF7E7F90028D9D10020EEE7FEF74F
:10535C00F3F9F8E703A8FFF773F80498F3E7684646
:10536C00FFF788F90198EEE7124B1B6813F0200F3A
:10537C0008D0104B1B68C3F3C1030F48D840E2E7B9
:10538C000E48BCE70C48BAE70120CFE70120CDE777
:10539C000120CBE70120C9E70120C7E70120C5E7C1
:1053AC000120C3E70120C1E70120BFE7505F0008DF
:1053BC00FFFC0F00004402580090D00300093D0090
:1053CC00836A13F0080F06D00268536823F4004375
:1053DC00816B0B435360836A13F0010F06D0026894
:1053EC00536823F40033C16A0B435360836A13F090
:1053FC00020F06D00268536823F48033016B0B4311
:10540C005360836A13F0040F06D00268536823F4C8
:10541C008023416B0B435360836A13F0100F06D04B
:10542C000268936823F48053C16B0B439360836AC7
:10543C0013F0200F06D00268936823F40053016C1C
:10544C000B439360836A13F0400F0AD002685368D1
:10545C0023F48013416C0B435360436CB3F5801FF2
:10546C000BD0836A13F0800F06D00268536823F4C4
:10547C000023C16C0B43536070470268536823F4DC
:10548C00C003816C0B435360EBE72DE9F8430546F1
:10549C000E4617469946DDF820802C68E46936EAFA
:1054AC0004030CBF01240024BC423AD1B8F1FF3FE5
:1054BC00F3D0FCF705F8A0EB0900404534D8B8F15F
:1054CC00000F33D02B681A6812F0040FE5D0B6F138
:1054DC00400218BF0122802EDFD0002ADDD0DA690D
:1054EC0012F0080F11D1DA6912F4006FD5D04FF415
:1054FC0000621A622846FFF7D7F92023C5F89030CE
:10550C00002385F8843003200CE008241C62284614
:10551C00FFF7CAF9C5F89040002385F884300120C4
:10552C0000E00020BDE8F8830320FBE70320F9E747
:10553C0030B583B004460023C0F89030FBF7C0FFB1
:10554C00054623681B6813F0080F10D123681B68ED
:10555C0013F0040F28D12023C4F88830C4F88C3001
:10556C000020E066206784F8840003B030BD6FF043
:10557C007E430093034600224FF400112046FFF7B0
:10558C0084FF0028E2D0226852E8003F23F0800319
:10559C0042E800310029F6D12023C4F888300023DA
:1055AC0084F884300320E0E76FF07E4300932B46B1
:1055BC0000224FF480012046FFF767FF0028CAD075
:1055CC00226852E8003F23F4907342E8003100292E
:1055DC00F6D1226802F1080353E8003F23F00103DF
:1055EC00083242E800310029F3D12023C4F88C3072
:1055FC00002384F884300320B7E778B310B5044651
:10560C00D0F888300BB32423C4F888302268136890
:10561C0023F001031360A36AE3B92046FFF76CFB88
:10562C00012811D02268536823F4904353602268F8
:10563C00936823F02A0393602268136843F00103F4
:10564C0013602046FFF774FF10BD80F88430FBF721
:10565C0055FED8E72046FFF7B3FEDEE70120704782
:10566C00436E2BB90123A0F86A30A0F8683070475C
:10567C0030B403689A68C2F342629968490F094DC5
:10568C006B5C1B01084C615C93FBF1F3A0F86A3076
:10569C00AB5C1B01A25C93FBF2F3A0F8683030BC4E
:1056AC00704700BF705F0008685F00087047704764
:1056BC00704790F88430012B18D0012380F8843087
:1056CC002423C0F8883003681A68196821F0010196
:1056DC00196022F000520023436601680A60202200
:1056EC00C0F8882080F88430184670470220704734
:1056FC0038B590F88430012B1DD00446012380F876
:10570C0084302423C0F8883003681D681A6822F09E
:10571C0001021A600268936823F060431943916098
:10572C00FFF79EFF23681D602023C4F888300020FB
:10573C0084F8840038BD0220FCE738B590F884303A
:10574C00012B1DD00446012380F884302423C0F89B
:10575C00883003681D681A6822F001021A6002681A
:10576C00936823F0606319439160FFF779FF236816
:10577C001D602023C4F88830002084F8840038BDD4
:10578C000220FCE738B51B4C4FF488752A460021E3
:10579C00204600F0D5FA2A460021601900F0D0FA14
:1057AC002A46002104F5087000F0CAFA2A460021A6
:1057BC0004F54C7000F0C4FA2A46002104F5886008
:1057CC0000F0BEFA2A46002104F5AA6000F0B8FAEF
:1057DC00012323800022628084F8583084F83C3006
:1057EC00054BC4F8B030054BC4F8B430044BC4F8C6
:1057FC00B83038BD90050024000048410000F0414D
:10580C000000204190F8583013B18B78332B00D026
:10581C00704710B4CA780C79002364F307034C79F1
:10582C0064F30F238C7964F31743C97961F31F6315
:10583C00512A57D8DFE812F0520058005D00620080
:10584C0067006C00710076007B00800086008C0085
:10585C00920098009E00A400AA00B000B600BC0004
:10586C00C200C800CE00D400DA00E000E600EC0074
:10587C00F200F800FE0004010A01100116011C01DF
:10588C00220156005600560056005600560056008F
:10589C0056005600560056005600560028012E01A0
:1058AC0034013A014001460156005600560056009C
:1058BC00560056005600560056005600560056002C
:1058CC00560056005600560056005600560056001C
:1058DC0056005600560056004C015201C365022377
:1058EC0080F8583010BC70470366032380F858309A
:1058FC00F8E74366042380F85830F3E78366052302
:10590C0080F85830EEE7C366062380F85830E9E794
:10591C000367072380F85830E4E74367082380F8CF
:10592C005830DFE78367092380F85830DAE7C3671C
:10593C000A2380F85830D5E7C0F880300B2380F864
:10594C005830CFE7C0F884300C2380F85830C9E7C2
:10595C00C0F888300D2380F85830C3E7C0F88C307D
:10596C000E2380F85830BDE7C0F890300F2380F834
:10597C005830B7E7C0F89430102380F85830B1E7AE
:10598C00C0F89830112380F85830ABE7C0F89C3041
:10599C00122380F85830A5E7C0F8A030132380F804
:1059AC0058309FE7C0F8A430142380F8583099E79A
:1059BC00C0F8A830152380F8583093E7C0F8AC3005
:1059CC00162380F858308DE7C0F8B030172380F8D4
:1059DC00583087E7C0F8B430182380F8583081E786
:1059EC00C0F8B830192380F858307BE7C0F8BC30C9
:1059FC001A2380F8583075E7C0F8C0301B2380F8A4
:105A0C0058306FE7C0F8C4301C2380F8583069E771
:105A1C00C0F8C8301D2380F8583063E7C0F8CC308C
:105A2C001E2380F858305DE7C0F8D0301F2380F873
:105A3C00583057E7C0F8D430202380F8583051E75D
:105A4C00C0F8D830212380F858304BE7C0F8DC3050
:105A5C00222380F8583045E7C0F8E030232380F843
:105A6C0058303FE7C0F8E430242380F8583039E749
:105A7C00C0F8E830252380F8583033E7C0F8EC3014
:105A8C00262380F858302DE7C0F8F030272380F813
:105A9C00583027E7C0F8F430282380F8583021E735
:105AAC00C0F8F830292380F858301BE7C0F8FC30D8
:105ABC002A2380F8583015E7C0F800312B2380F8E2
:105ACC0058300FE7C0F804312C2380F8583009E720
:105ADC00C0F808312D2380F8583003E7C0F80C319A
:105AEC00002380F85830FDE610B584B000230193F4
:105AFC00029301AA0DF10E010848FBF77DF9BDF8E0
:105B0C000E300BB104B010BD054C01A9204600F0BD
:105B1C002DF801A92046FFF775FEF3E75804002481
:105B2C009005002400234365036503644364836488
:105B3C00C3647047F8B507460C461E461046FAF784
:105B4C00E3FB05463846FAF795FC2946FAF7E6FCDE
:105B5C0005460120B0400138FAF78CFC0146284676
:105B6C00FAF790FD2146FAF7D1FBF8BDF8B50446DB
:105B7C000D460B7803F00F0343600B781B09836011
:105B8C004B78887840EA0320E060CB780F793F09A6
:105B9C0047EA031727610E79360206F470664B79D3
:105BAC001E436661D4F8B02002F100411023FFF7C8
:105BBC00C1FF2062D4F8B42002F100410C23384616
:105BCC00FFF7B8FF6062D4F8B82002F100410C2353
:105BDC003046FFF7AFFFA062A879FAF747FC606385
:105BEC00E879FAF743FCA063F8BD00B583B0114423
:105BFC00FF238DF800308DF801308DF802308DF8D0
:105C0C0003308DF804308DF805308DF80630FD2307
:105C1C008DF8073008236A4689B2FBF7AEF803B05B
:105C2C005DF804FB10B50C4691F83C30013B032B9E
:105C3C0007D8DFE803F0020A101600220988FFF7E4
:105C4C00D4FF2046FFF76EFF10BD4FF48072098819
:105C5C00FFF7CBFFF5E74FF400720988FFF7C5FF9C
:105C6C00EFE74FF440720988FFF7BFFFE9E7000048
:105C7C0010B582B000F00F04C0F303108DF8004093
:105C8C008DF8010055208DF802008DF803108DF869
:105C9C0004208DF805309DF810308DF806309DF8F5
:105CAC0014308DF8073008236A4640F2FF71024821
:105CBC00FBF763F802B010BD5804002400B583B0A4
:105CCC0000F00F03C0F303108DF804308DF80500BD
:105CDC00AA238DF8063001238DF8073004230DEB31
:105CEC00030240F2FF710348FBF747F803B05DF87D
:105CFC0004FB00BF5804002470B50D4E0D4D761BEF
:105D0C00B61006D0002455F8043B01349847A6423F
:105D1C00F9D1094E094D761B00F0D2F8B61006D019
:105D2C00002455F8043B01349847A642F9D170BDC4
:105D3C00845F0008845F00088C5F0008845F0008A3
:105D4C00F0B4860746D0541E002A3CD0CAB2034693
:105D5C0001E0013C37D303F8012B9D07F9D1032C4B
:105D6C002AD9CDB245EA05250F2C45EA054534D98B
:105D7C00A4F1100222F00F0C03F12007160967445E
:105D8C0003F1100242E9045542E902551032BA42BD
:105D9C00F8D1721C14F00C0F03EB021204F00F0676
:105DAC0013D0331F23F003030433134442F8045B72
:105DBC009342FBD106F003042CB1CAB21C4403F885
:105DCC00012B9C42FBD1F0BC704734461346002C8F
:105DDC00F3D1F8E714460346C1E71A462646E0E736
:105DEC00024B13B1024800F005B8704700000000E8
:105DFC000D5E0008002301461A46184600F01AB83A
:105E0C0038B5084B084D5B1B9C1007D0043B1D4458
:105E1C00013C55F804399847002CF9D1BDE83840BD
:105E2C0000F054B8905F00088C5F0008704700BF0A
:105E3C00704700BF2DE9F047DFF880A00646DAF87E
:105E4C00000098460F469146FFF7F0FF1A4B1B686F
:105E5C00D3F8484124B365681F2D26DC5EB9AB1C12
:105E6C000135DAF80000656044F82370FFF7E0FFB5
:105E7C000020BDE8F08704EB85030121C3F888906E
:105E8C00D4F88821A9400A43022EC4F88821C3F80B
:105E9C000881E4D1D4F88C311943C4F88C11DEE7B5
:105EAC0003F5A674C3F84841D5E7DAF80000FFF70C
:105EBC00BFFF4FF0FF30DCE7785F000838040024A8
:105ECC00F8B500BFF8BC08BC9E467047F8B500BFDB
:085EDC00F8BC08BC9E467047AB
:105EE40000000000000000000000000000000000AE
:105EF4000000000001000000020000000300000098
:105F04000400000000000000050000000000000084
:105F14000000000000000000060000000000000077
:105F24000000000000000000070000000000000066
:105F34000102030401020304060708090001020325
:105F440004050607080C1014182030400100020054
:105F54000400060008000A000C00100020004000A5
:105F64008000000108040204080101010101010389
:085F74000701000010000024E9
:085F7C00BCA8FF7F010000003A
:085F8400ED5D0008F1020008C8
:045F8C00CD0200083A
:105F90000090D0030090D00301000000100000002A
:105FA00000000000FC02002464030024CC03002451
:105FB00000000000000000000000000000000000E1
:105FC00000000000000000000000000000000000D1
:105FD00000000000000000000000000000000000C1
:105FE00000000000000000000000000000000000B1
:105FF00000000000000000000000000000000000A1
:106000000000000000000000000000000000000090
:106010000000000000000000000000000000000080
:106020000000000000000000000000000000000070
:106030000000000000000000000000000000000060
:10604000000000000000000001000000000000004F
:106050000E33CDAB34126DE6ECDE05000B00000014
:106060000000000000000000000000000000000030
:106070000000000000000000000000000000000020
:106080000000000000000000000000000000000010
:106090000000000000000000000000000000000000
:0C63C0000000000000000000301000246D
:04000005080013B527
:00000001FF
